:0200000480007A
:100000006F00C004732F2034930F8000630AFF0336
:10001000930F90006306FF03930FB0006302FF038A
:10002000170F0080130F0FFE63040F0067000F000F
:10003000732F203463540F006F00400093E19153FD
:10004000171F000023203FFC6FF09FFF732540F136
:1000500063100500970200009382020173905230F2
:10006000735000189702000093820202739052307E
:10007000B70200809382F2FF7390023B9302F0017B
:100080007390023A9702000093828201739052307B
:100090007350203073503030735040309301000063
:1000A00097020000938242F67390523013051000BD
:1000B0001315F501634C05000F00F00F93011000BC
:1000C0009308D0051305000073000000970200801C
:1000D000938242F3638E020073905210B7B2000015
:1000E000938292107390223073232030E39862F44D
:1000F00073500030970200009382420173901234D3
:10010000732540F173002030B70001FF938000F0A9
:1001100037110F0F1301F1F033E72000B70E10FF76
:10012000938EFEF0930120006312D74BB710F00FAF
:10013000938000FF37F1F0F01301010F33E7200047
:10014000B70EF1FF938E0EFF930130006310D74975
:10015000B700FF009380F00F37110F0F1301F1F07C
:1001600033E72000B71EFF0F938EFEFF9301400080
:10017000631ED745B7F00FF09380F00037F1F0F031
:100180001301010F33E72000B7FEFFF0938EFE0F3F
:1001900093015000631CD743B70001FF938000F028
:1001A00037110F0F1301F1F0B3E02000B70E10FF6D
:1001B000938EFEF093016000639AD041B70001FF77
:1001C000938000F037110F0F1301F1F033E120009D
:1001D000B70E10FF938EFEF0930170006318D13FAD
:1001E000B70001FF938000F0B3E01000B70E01FFED
:1001F000938E0EF093018000639AD03D13020000AD
:10020000B70001FF938000F037110F0F1301F1F0D9
:1002100033E72000130307001302120093022000AB
:10022000E31052FEB70E10FF938EFEF09301900084
:10023000631ED33913020000B710F00F938000FF44
:1002400037F1F0F01301010F33E720001300000035
:10025000130307001302120093022000E31E52FC56
:10026000B70EF1FF938E0EFF9301A0006310D337FA
:1002700013020000B700FF009380F00F37110F0F3B
:100280001301F1F033E72000130000001300000019
:10029000130307001302120093022000E31C52FC18
:1002A000B71EFF0F938EFEFF9301B0006310D33390
:1002B00013020000B70001FF938000F037110F0F09
:1002C0001301F1F033E72000130212009302200023
:1002D000E31252FEB70E10FF938EFEF09301C000A2
:1002E0006316D72F13020000B710F00F938000FFA2
:1002F00037F1F0F01301010F1300000033E7200085
:100300001302120093022000E31052FEB70EF1FF19
:10031000938E0EFF9301D000631AD72B13020000B7
:10032000B700FF009380F00F37110F0F1301F1F0AA
:10033000130000001300000033E720001302120036
:1003400093022000E31E52FCB71EFF0F938EFEFFA8
:100350009301E000631CD72713020000B70001FFE0
:10036000938000F01300000037110F0F1301F1F01C
:1003700033E720001302120093022000E31052FE24
:10038000B70E10FF938EFEF09301F0006310D72597
:1003900013020000B710F00F938000FF130000005D
:1003A00037F1F0F01301010F1300000033E72000D4
:1003B0001302120093022000E31E52FCB70EF1FF5D
:1003C000938E0EFF930100016312D72113020000E8
:1003D000B700FF009380F00F13000000130000002F
:1003E00037110F0F1301F1F033E720001302120051
:1003F00093022000E31E52FCB71EFF0F938EFEFFF8
:10040000930110016314D71D1302000037110F0F61
:100410001301F1F0B70001FF938000F033E72000F3
:100420001302120093022000E31252FEB70E10FFD7
:10043000938EFEF093012001631AD7191302000076
:1004400037F1F0F01301010FB710F00F938000FFA8
:100450001300000033E72000130212009302200073
:10046000E31052FEB70EF1FF938E0EFF93013001A1
:10047000631ED7151302000037110F0F1301F1F09F
:10048000B700FF009380F00F13000000130000007E
:1004900033E720001302120093022000E31E52FCF7
:1004A000B71EFF0F938EFEFF930140016310D71319
:1004B0001302000037110F0F1301F1F013000000B9
:1004C000B70001FF938000F033E720001302120011
:1004D00093022000E31052FEB70E10FF938EFEF041
:1004E000930150016314D70F1302000037F1F0F0AD
:1004F0001301010F13000000B710F00F938000FFED
:100500001300000033E720001302120093022000C2
:10051000E31E52FCB70EF1FF938E0EFF93016001B4
:100520006316D70B1302000037110F0F1301F1F000
:100530001300000013000000B700FF009380F00FCD
:1005400033E720001302120093022000E31E52FC46
:10055000B71EFF0F938EFEFF930170016318D7073C
:10056000B70001FF938000F033611000B70E01FF68
:10057000938E0EF093018001631AD105B700FF003E
:100580009380F00F33E10000B70EFF00938EFE0F53
:1005900093019001631CD103B3600000930E00002F
:1005A0009301A0016394D003B7101111938010112F
:1005B000372122221301212233E02000930E000074
:1005C0009301B0016314D001631030020F00F00FEB
:1005D000638001009391110093E111009308D0050D
:1005E00013850100730000000F00F00F930110004D
:1005F0009308D0051305000073000000731000C0BD
:0406000000000000F6
:1010000000000000000000000000000000000000E0
:1010100000000000000000000000000000000000D0
:1010200000000000000000000000000000000000C0
:1010300000000000000000000000000000000000B0
:081040000000000000000000A8
:040000058000000077
:00000001FF
